:020000040000FA
:0400000080317928AA
:100008007E1480310B1D09280A287728013020002A
:10001800C3070030C43D7A08F5007908F400F435C8
:10002800F50DF435F50D7408643EF6000030753DA5
:10003800F7007708803AF8004408803A7802031DF0
:1000480027284308760203182A282B285F2820002F
:10005800C301C4014535203E86008701403FF400B6
:10006800413FF50074087B07840075087C3D8500D6
:1000780000089E319F2680319E310D268031200058
:100088008E168E120130FB070030FC3D4535203EB0
:1000980086008701403FF400413FF50074087B0764
:1000A800840075087C3D85001200031D5C285D28CE
:1000B8005F28FB01FC0120008C1E63286428762839
:1000C8004208803AF40080307402031D6D28013024
:1000D8004102031C702871287628FF302000C107D0
:1000E800FF30C23D0B117E10090080317B28CD30D6
:1000F80084009D308500203086000030870018304D
:100108009D31C7258031F901FA01FB01FC01C101CC
:10011800C201C301C401C501C6017E1020009E3181
:100128003B2E4C346F34723465346D34203469346A
:100138007034733475346D34203464346F346C34F3
:100148006F34723420347334693474342034613435
:100158006D34653474342C34203463346F346E3425
:100168007334653463347434653474347534723478
:1001780020346134643469347034693473346334DA
:1001880069346E346734203465346C3469347434BB
:100198002C342034733465346434203464346F343C
:1001A800203465346934753473346D346F34643491
:1001B8002034743465346D3470346F3472342034C0
:1001C80069346E346334693464346934643475343E
:1001D8006E34743420347534743420346C3461349F
:1001E80062346F34723465342034653474342034A6
:1001F80064346F346C346F347234653420346D3445
:10020800613467346E346134203461346C34693459
:100218007134753461342E342034543465346C347C
:100228006C347534733420346D346F346C34653405
:10023800733474346934653420346E3475346E34F0
:10024800633420346E346F346E34203462346C344A
:1002580061346E3464346934743420346D346134F8
:10026800733473346134203465346E3469346D34D6
:1002780020346E346534633420346434753469341E
:1002880020346E3475346E3463342E34203446345E
:1002980061346D346534733420346134633420340C
:1002A800743475347234703469347334203465347A
:1002B800673465347334743461347334203473347C
:1002C800653464342034743465346D347034753472
:1002D80073342034753472346E3461342E342034DF
:1002E8004C3469346234653472346F342034653484
:1002F8006E3469346D342034733465346434203496
:1003080066346134753463346934623475347334F3
:10031800203474347534723470346934733420344E
:1003280069346E342E34203445346C3465346D347D
:1003380065346E34743475346D34203469346E34F5
:1003480074346534673465347234203465346E34FB
:1003580069346D3420346E346534713475346534E1
:10036800203476346F346C347534743470346134BA
:1003780074342034613463342034743469346E3412
:1003880063346934643475346E34743420347634A8
:1003980069347434613465342E34203449346D340E
:1003A8007034653472346434693465347434203498
:1003B8006E3475346C346C34613420346D3461348B
:1003C8006C34653473347534613464346134203486
:1003D800703465346C346C3465346E34743465341C
:1003E8007334713475346534203465346C3469344D
:1003F8007434203465346734653474342034673495
:10040800723461347634693464346134203463344A
:1004180075346D34203473346F346334693469341B
:1004280073342E3420345634693476346534723457
:10043800723461342034613464346934703469341A
:100448007334633469346E346734203461347434FB
:10045800203469346E342034743465346C346C342C
:1004680075347334203469346E34743465346734C5
:1004780065347234203466346534753467346934CD
:100488006134743420347334633465346C346534C3
:100498007234693473347134753465342E342034CD
:1004A80055347434203465346E3469346D342034F2
:1004B80062346C3461346E34643469347434203496
:1004C80076346F346C347534743470346134743405
:1004D80020346D3461346534633465346E3461348A
:1004E8007334203476346F346C3475347434703427
:1004F800613474342E34203444346F346C346F34A3
:10050800723420346D346F34723462346934203478
:100518006E346F346E34203461347234633475341D
:10052800203472346934733475347334203471343C
:1005380075346934733420347634613472346934F0
:100548007534733420347134753461346D34203427
:1005580071347534693473347134753465342034C6
:10056800693464342E342034553472346E34613432
:1005780020346E34653463342034743469346E3412
:1005880063346934643475346E34743420347034AC
:10059800723461346534733465346E3474342034A1
:1005A800733465346D347034653472342034663491
:1005B80065347534673469346134743420346E3486
:1005C8006934623468342E342034453467346534F1
:1005D800733474346134733420347334653464345C
:1005E8002034733465346434203472346934733499
:1005F8007534733420347034723465347434693427
:1006080075346D342E342034543469346E34633484
:100618006934643475346E347434203474346F340B
:10062800723474346F347234203461346C34693405
:100638007134753461346D3420346E3475346C34EF
:100648006C346134203466346134633469346C3416
:1006580069347334693420346334723461347334E4
:1006680020346634653472346D3465346E347434D1
:1006780075346D3420346F34643469346F34203405
:1006880065347534203466346534753467346934B8
:10069800613474342E3420344434693467346E340D
:1006A80069347334733469346D34203465346E348A
:1006B80069346D34203473346934743420346134CB
:1006C8006D34653474342034763465346E3465346E
:1006D8006E3461347434693473342034753472344C
:1006E8006E34613420346334753472347334753441
:1006F80073342034653467346534743420346E348C
:1007080075346E3463342E342034503475346C347C
:10071800763469346E346134723420346D34613423
:10072800743474346934733420346E3475346E34EC
:1007380063342034733465346434203462346C3464
:1007480061346E3464346934743420346C346934FC
:100758006234653472346F34203476346F346C34D8
:1007680075347434703461347434203473346534BB
:1007780064342E3420344D34613467346E3461343B
:1007880020346634723469346E34673469346C34B6
:100798006C3461342034753472346E3461342034EE
:1007A80070346F34723474347434693474346F341C
:1007B80072342034723468346F346E346334753470
:1007C8007334203464346F346C346F3472342034AE
:1007D8007034753472347534733420346E346F3435
:1007E8006E34203465346E3469346D34203470349A
:1007F800723461346534733465346E3474342E3431
:100808002034413464346934703469347334633463
:1008180069346E346734203476346934743461341E
:1008280065342034703472346F3469346E34203453
:1008380073346134673469347434743469347334A8
:1008480020346E34693473346C3420347234683430
:100858006F346E3463347534733420346D346134DA
:1008680074347434693473342034723468346F34B3
:100878006E346334753473342034753472346E34A2
:1008880061342E3420344E3475346C346C34613415
:10089800203466346134633469346C3469347334B5
:1008A800693420346D346F347234623469342034DE
:1008B800743465346D347034753473342034693469
:1008C8006134633475346C3469347334203475346A
:1008D80072346E34613420346934643420347634AC
:1008E8006F346C3475347434703461347434203437
:1008F8006C3461346334753473342E34203450349A
:1009080068346134733465346C346C3475347334DE
:10091800203476346534733474346934623475340D
:100928006C3475346D3420346C346F3472346534FF
:100938006D3420347334653464342034723469344B
:10094800733475347334203475346C3474347234BD
:1009580069346334693465347334203474347234DC
:1009680069347334743469347134753465342034BB
:100978006E3475346C346C3461342E342034543411
:100988006F34723474346F3472342034693464349C
:10099800203461346C34693471347534653474349A
:1009A80020346C34653463347434753473342034CF
:1009B800703472346F3469346E3420346E34693470
:1009C8006234683420346E34693473346C342034BF
:1009D80063346F346E34643469346D3465346E3422
:1009E800743475346D342034693464342E340034EE
:1009F80041346C346934713475346534743420345A
:100A080073346134673469347434743469347334D6
:100A1800203469346434203463346F346E3473346E
:100A28006534633474346534743475347234203402
:100A3800703475347234753473342E34203452342F
:100A480068346F346E3463347534733420346D34E1
:100A580061347434743469347334203472346834CF
:100A68006F346E34633475347334203475347234AF
:100A78006E34613420346E346534713475346534C1
:100A8800203476346934763465347234723461349F
:100A980020346A347534733474346F342E3420340B
:100AA8004E34653474347534733420346534743496
:100AB80020346D3461346C34653473347534613486
:100AC800643461342034663461346D34653473348D
:100AD800203461346334203474347534723470349F
:100AE800693473342034653467346534733474344A
:100AF800613473342E3420344D3461347534723497
:100B080069347334203475346C3474347234693411
:100B18006334653473342034653472346F34733419
:100B2800203469346E342034633475347234733449
:100B380075347334203474347534723470346934D1
:100B4800733420346D346134733473346134203435
:100B5800743469346E3463346934643475346E348F
:100B6800743420346434753469342E342034463473
:100B78006134633469346C346934733469342034CF
:100B88006D346F34723462346934203474346534AB
:100B98006D3470347534733420346934613463349B
:100BA80075346C34693473342034753472346E346B
:100BB8006134203469346434203476346F346C34CE
:100BC8007534743470346134743420346C34613462
:100BD80063347534733420346C3461346F34723454
:100BE80065346534743420346E346F346E342E3486
:100BF8002034503468346134723465347434723457
:100C0800613420346434693461346D34203473348D
:100C180069347434203461346D3465347434203468
:100C28006E34693473346C342034733475347334EB
:100C3800633469347034693474342034613464340E
:100C48006934703469347334633469346E346734A6
:100C5800203462346934623465346E3464347534F3
:100C68006D3420346534733474342E3420344E3467
:100C780061347334633465347434753472342034B5
:100C88007234693464346934633475346C3475345B
:100C9800733420346D347534733420346D346134D6
:100CA8007534723469347334203476346934743466
:100CB80061346534203475346C3474347234693476
:100CC800633469346534733420346C3465346F3478
:100CD800203469346E34743465346734653472345E
:100CE80020346D3461346C34653473347534613454
:100CF8006434613420346E3475346E3463342E3485
:100D080020344534743420346E3465347434753486
:100D1800733420346534743420346D3461346C3465
:100D28006534733475346134643461342034663422
:100D380061346D3465347334203461346334203461
:100D480074347534723470346934733420346534CF
:100D580067346534733474346134733420347334D1
:100D6800653464342E34203443346F346E3467343D
:100D7800753465342034713475346934733471349E
:100D880075346534203465346734653473347434A9
:100D98006134733420346434693461346D342034FC
:100DA80069346E34203461347234633475342034D9
:100DB8006334753472347334753473342E34203498
:100DC8004634613475346334693462347534733449
:100DD800203469346E3420346F3472346E346134A4
:100DE8007234653420347134753461346D34203490
:100DF80076346934763465347234723461342E341E
:100E0800203444346F346E346534633420346D34A4
:100E1800613473347334613420347334613470341E
:100E2800693465346E34203466346134753463341F
:100E3800693462347534733420346534743420343E
:100E48006D346F346C346534733474346934653498
:100E58002E34203443347534723473347534733417
:100E680020347434753472347034693473342034F3
:100E78006D346134733473346134203474346934B8
:100E88006E3463346934643475346E3474342034A5
:100E98006434753469342034753474342E34203411
:100EA800533465346D3470346534723420346134AD
:100EB8007534633474346F34723420346E3465346A
:100EC800713475346534203476346934743461345B
:100ED80065342034743465346D3470347534733447
:100EE80020347134753461346D3420347034653491
:100EF8006C346C3465346E347434653473347134E2
:100F08007534653420346E346534633420346E347B
:100F180061346D34203461346C346934713475341F
:100F280061346D342E3420345534743420346D34A7
:100F38006F347234623469342034743469346E34F2
:100F480063346934643475346E34743420346134F1
:100F58007534673475346534203469346E347434C8
:100F680065347234643475346D342E3420344E3420
:100F780065347434753473342034653474342034EF
:100F88006D3461346C34653473347534613464346D
:100F980061342034663461346D34653473342034FC
:100FA800613463342E3420345634693474346134F3
:100FB80065342034743465346D3470347534733466
:100FC80020347134753461346D34203470346534B0
:100FD8006C346C3465346E34743465347334713401
:100FE8007534653420346E346534633420346E349B
:100FF80061346D342E34203445346E3469346D34A4
:1010080020346E3475346C346C346134203461347B
:101018006C34693471347534653474342034703404
:101028006F34723474347434693474346F34723491
:1010380020346C34613463347534733420346C3444
:1010480075346334743475347334203461346334E0
:10105800633475346D34733461346E3420347434CD
:101068006F34723474346F347234203470346F34A3
:1010780073347534653472346534203461346334C0
:101088002E3420344134723463347534203472344D
:101098006934733475347334203471347534693475
:1010A800733420347634613472346934753473346B
:1010B80020347134753461346D342E3420344C341A
:1010C80065346F34203461342034643469346134D5
:1010D8006D34203473346F346C346C346934633455
:1010E800693474347534643469346E342034743437
:1010F80065346D3470346F34723420346934643438
:1011080020346534753420346E34693473346C3467
:1011180020346E3475346E3463342E3420344934BC
:101128006434203466346134753463346934623429
:101138007534733420346E34693473346C34203429
:10114800743469346E3463346934643475346E3499
:1011580074342034653467346534743420346E3420
:1011680075346C346C3461346D3420346E346F34BF
:101178006E3420346E346934733469342E34003458
:1011880046346534753467346934613474342034D2
:1011980076346934763461346D347534733420347C
:1011A800613474342034613475346734753465348B
:1011B80020346534673465347434203461347234CF
:1011C8006334753420346434693463347434753466
:1011D8006D342E34203450346F34733475346534A0
:1011E8007234653420346D346F3472346234693447
:1011F80020346C3465346F342034753472346E3472
:10120800613420346D346F346C3465347334743421
:1012180069346534203461347434203465346C3472
:1012280065346D3465346E34743475346D342034FB
:10123800653475342E34203443346F346E34673457
:101248007534653420346D346134753472346934DE
:1012580073342034723468346F346E3463347534C4
:1012680073342034613465346E34653461346E34DB
:101278002034763465346C34203465346C34693405
:1012880074342E3420344534753420347334653442
:101298006D34203469346E3474346534673465349D
:1012A80072342034763469347434613465342034CB
:1012B8006A347534733474346F3420346534673465
:1012C800653474342E3420344F34723463346934C2
:1012D80020346534753420346C346F3462346F34A0
:1012E8007234743469347334203465346C3465343E
:1012F8006D3465346E34743475346D3420346E3422
:101308006934623468342E342034413420346434EF
:10131800693461346D34203473346F346C346C3414
:1013280069346334693474347534643469346E34BC
:101338002034743465346D3470346F34723420342E
:101348006934643420346534753420346E34693437
:1013580073346C342E34203443346F346E34643434
:1013680069346D3465346E34743475346D342034B6
:101378006D346134743474346934733420347034A3
:1013880065346C346C3465346E3474346534733459
:1013980071347534653420346934643420346E34DF
:1013A8006934623468342E342034563465346C34ED
:1013B800203465346C3469347434203473346334C1
:1013C80065346C346534723469347334713475340B
:1013D800653420346D34613475347234693473344F
:1013E8002034703465346C346C3465346E34743441
:1013F800653473347134753465342E34203456347E
:101408006F346C347534743470346134743420340B
:101418006D3461346534633465346E3461347334E7
:10142800203476346F346C347534743470346134E9
:101438007434203462346C3461346E346434693406
:101448007434203461346C346934713475346134E3
:101458006D34203465347434693461346D34203427
:1014680065347234613474342034763465346C34C1
:10147800693474342E34203450346834613472340E
:10148800653474347234613420346D3461346734B3
:101498006E346134203461346334203470346C34F5
:1014A800613463346534723461347434203476348E
:1014B8006534733474346934623475346C34753417
:1014C8006D3420346C346534633474347534733457
:1014D80020346D3461347534723469347334203493
:1014E80075346C34743472346934633465347334E9
:1014F8002E34203456346934763465347234723478
:1015080061342034733475347334703465346E3414
:1015180064346934733473346534203470346F340C
:10152800743465346E347434693420346E347534EC
:101538006C346C3461346D34203461346334203459
:1015480074346F34723474346F34723420347634B3
:1015580069347434613465342034703475347234C9
:1015680075347334203466346134753463346934C3
:101578006234753473342E34203455347434203442
:10158800763465346E3465346E3461347434693459
:1015980073342034743465346C346C347534733477
:1015A800203469346E3420346D34653474347534C1
:1015B80073342034763475346C3470347534743440
:1015C80061347434653420346534753420347334AC
:1015D800633465346C34653472346934733471340B
:1015E800753465342034663465346C346934733446
:1015F800203469346D347034653472346434693439
:10160800653474342E34203449346E3420346834CC
:1016180065346E34643472346534723469347434C5
:101628002034673472346134763469346434613414
:101638002034723475347434723475346D34203413
:1016480071347534693473347134753465342034C5
:101658006E346F346E342034743465346C346C34C6
:101668007534733420346F347234633469342034FD
:10167800613463342E3420344D346134743474341A
:10168800693473342034703465346C346C346534A4
:101698006E3474346534733471347534653420347D
:1016A8006934643420346E346934623468342034E4
:1016B80074346F34723474346F347234203469344F
:1016C8006434203461346C3469347134753465346D
:1016D800743420346C34653463347434753473343E
:1016E8002E3420344534743420346E3465347434E4
:1016F8007534733420346534743420346D34613473
:101708006C34653473347534613464346134203432
:10171800663461346D34653473342E342034453482
:1017280073347434203475346C34743472346934DA
:101738006334693465347334203469346E347434F2
:1017480065346734653472342034713475346934DF
:101758007334203461347534633474346F347234C0
:10176800203465346C34693474342034733465340B
:1017780064342E342034503465346C346C3465341D
:101788006E3474346534733471347534653420348C
:10179800733469347434203461346D34653474348A
:1017A800203470346F34723474347434693474345B
:1017B8006F347234203465346734653474342E34AD
:1017C80020344E3475346E346334203465346734D1
:1017D8006534743420346C346F34723465346D3449
:1017E800203464346F346C346F347234203473347E
:1017F800653464342034763469347634653472342C
:1018080072346134203469347034733475346D340F
:1018180020346E3475346E3463342E3420345034AE
:1018280065346C346C3465346E34743465347334B4
:10183800713475346534203465346C3469347434E7
:101848002034653467346534743420346734723432
:1018580061347634693464346134203463347534E3
:101868006D34203473346F346334693469347334B9
:1018780020346E34613474346F34713475346534A3
:101888002034703465346E346134743469346234AD
:101898007534733420346534743420346D346134D1
:1018A80067346E34693473342E34003455347434E8
:1018B800203474346F34723474346F347234203496
:1018C8007034723465347434693475346D3420344A
:1018D8007634693476346534723472346134203441
:1018E800733475347334703465346E3464346934E5
:1018F800733473346534203470346F34743465341D
:101908006E34743469342E34203449346E3474346B
:10191800653467346534723420346D3461346C3422
:1019280065347334753461346434613420346E340E
:1019380075346E3463342034763465346C34203432
:1019480072346934733475347334203463346F34C7
:101958006D346D346F3464346F34203476346934C4
:101968007634653472347234613420346D346134C1
:101978006534633465346E346134733420346134CF
:101988006334633475346D34733461346E342034A5
:101998006C3461346334753473342E3420344E34EB
:1019A8006F346E3420347134753461346D342034BE
:1019B8006C3461346334753473342034733475345F
:1019C8007334703465346E34643469347334733406
:1019D8006534203466346134753463346934623470
:1019E80075347334203469346E3474346534723425
:1019F800643475346D34203470346F347334753412
:101A080065347234653420346C346F347234653420
:101A18006D34203469347034733475346D342E3435
:101A28002034533461346734693474347434693419
:101A38007334203465347534203476346F346C3420
:101A48007534743470346134743420346F346434CD
:101A580069346F34203466346134633469346C34E7
:101A6800693473346934733420346D3461347534B3
:101A78007234693473342E34203443346F346E3402
:101A8800643469346D3465346E34743475346D344B
:101A980020347634693474346134653420347334D2
:101AA80061347034693465346E342034703465348C
:101AB8006C346C3465346E34743465347334713416
:101AC800753465342034683461346234693474346C
:101AD80061346E34743420346D346F34723462344B
:101AE8006934203474347234693473347434693426
:101AF8007134753465342E34203456346934743472
:101B08006134653420347334753473346334693420
:101B18007034693474342034743465346C346C34FF
:101B28007534733420346D346134753472346934E7
:101B380073342034613420346434693461346D344E
:101B480020346D3461346534633465346E34613403
:101B580073342034733465346434203465346E341B
:101B680069346D342034753474342E34203441345F
:101B7800743420346C346534633474347534733499
:101B88002034753472346E346134203464347534DE
:101B980069347334203463346F346E34763461348A
:101BA8006C346C34693473342E3420344D346134DD
:101BB80067346E34613420347334693474342034B7
:101BC80061346D346534743420347034753472344F
:101BD800753473342034673472346134763469343C
:101BE80064346134203471347534693473342E3478
:101BF80020344D3461347334733461342034743494
:101C080069346E3463346934643475346E347434CE
:101C180020346E3475346E34633420347034753443
:101C28006C34763469346E346134723420347334ED
:101C380061347034693465346E34203465347434F6
:101C480020346C346934673475346C34613420342E
:101C580075346C346C3461346D3463346F3472347D
:101C68007034653472342E34203443346F346E3417
:101C7800643469346D3465346E34743475346D3459
:101C880020346D34613474347434693473342034DA
:101C9800703465346C346C3465346E347434653443
:101CA80073347134753465342034693464342034C1
:101CB8006E34693462346834203474346F34723466
:101CC80074346F34723420346934643420346134A9
:101CD8006C346934713475346534743420346C343C
:101CE8006534633474347534733420347034723426
:101CF8006F3469346E342E34203449346E342034D1
:101D08006E34693473346C3420346E34693473340B
:101D1800693420347334633465346C346534723414
:101D280069347334713475346534203465347534EA
:101D3800203475346C3474347234693463346534E3
:101D4800733420347634693474346134653420341F
:101D580061347534633474346F34723420346534C8
:101D680075342E3420344F3472346334693420345B
:101D78007334613467346934743474346934733453
:101D8800203465347534203476346F346C347534CB
:101D9800743470346134743420346F346434693486
:101DA8006F34203466346134633469346C34693494
:101DB80073346934733420346D3461347534723457
:101DC800693473342E3420344534743420346F34F9
:101DD800643469346F342034703465346C346C3452
:101DE80065346E34743465347334713475346534E1
:101DF80020346434693461346D34203476346F347B
:101E08006C3475347434703461347434203463340D
:101E18006F346D346D346F3464346F3420347334FC
:101E28006534643420346534673465347334743409
:101E380061347334203465346734653473347434EE
:101E48006134733420346634723469346E346734E0
:101E580069346C346C3461342E3420345334653432
:101E68006434203465346C3465346D3465346E34D0
:101E7800743475346D342034743465346D3470348E
:101E8800753473342034653467346534733474348A
:101E980061347334203473346534643420347334D7
:101EA800653464342034723469347334753473346B
:101EB8002E342034533469347434203461346D340E
:101EC800653474342034763465346E3465346E3455
:101ED80061347434693473342034753472346E3434
:101EE8006134203463347534723473347534733424
:101EF800203465346734653474342E3420344534E2
:101F08006E3469346D342034753474342034733449
:101F180065346D34203476346934763465347234FB
:101F280072346134203461346C34693471347534FA
:101F3800653474342034653467346534743420343B
:101F48007334693474342E34203444346F346E342A
:101F580065346334203461346434693470346934EA
:101F68007334633469346E346734203474347234AF
:101F78006934733474346934713475346534203495
:101F88007234693473347534733420346E34653480
:101F980063342034663465347534673469346134A5
:101FA8007434203469346E342034663465347234C1
:101FB8006D3465346E34743475346D342034703453
:101FC8006F34733475346534723465342E340034A8
:101FD8004434693461346D34203464346F346E347D
:101FE800653463342034613464346934703469345A
:101FF8007334633469346E3467342034743472341F
:102008006934733474346934713475346534203404
:102018007234693473347534733420346E346534EF
:1020280063342E342034563469347634653472344B
:1020380072346134203476346934743461346534EC
:10204800203463346F346E34673475346534203427
:1020580065347534203463346F346E3473346534C6
:102068007134753461347434203461346334203409
:10207800663465346C3469347334203464346F34B2
:102088006E346534633420346534743420346F34EA
:10209800643469346F342E3420344F3472346E34DF
:1020A8006134723465342034613472346334753485
:1020B80020346434753469342034763469347634A1
:1020C80061346D347534733420346134723463345C
:1020D80075342034663465346C34693473342E3482
:1020E8002034563469347634653472347234613449
:1020F80020346D3461346534633465346E3461344E
:102108007334203461346334633475346D34733418
:1021180061346E3420346C34613463347534733410
:102128002034763465346C34203466346134633456
:1021380069346C34693473346934733420347634D4
:102148006F346C34753474347034613474342034BE
:102158006534733474342034763465346C346934BB
:1021680074342034653467346534733474346134BA
:1021780073342E342034533465346D3470346534FC
:1021880072342034663465347534673469346134A4
:10219800743420346E3469346234683420347334CF
:1021A800653464342034703475346C34763469346E
:1021B8006E34613472342034703472346F3469345C
:1021C8006E3420346734723461347634693464345C
:1021D80061342E34203445347434203474346F34EC
:1021E800723474346F347234203463346F346E3420
:1021F800733465347134753461347434203469341B
:102208006434203470346F3472347434613420345C
:102218006E346934623468342034763465346E340C
:1022280065346E34613474346934733420346334FF
:1022380072346134733420347334653464342E3426
:10224800203445346C3465346D3465346E347434FC
:1022580075346D34203469346E34743465346734BD
:1022680065347234203465346E3469346D34203406
:102278006E346534713475346534203476346F3493
:102288006C3475347434703461347434203461348B
:1022980063342E34203452346934733475347334CF
:1022A800203461347434203475346C3474347234AA
:1022B800693463346534733420346D3469342034BC
:1022C800743465346D347034753473342E3420347A
:1022D8005634613472346934753473342034763446
:1022E80065346C3420347034683461347234653445
:1022F8007434723461342034763465346C34203468
:1023080074347534723470346934733420346E34F0
:1023180075346E346334203465346734653474340A
:102328002E34203449346E3420346D34653474349A
:10233800753473342034763475346C3470347534B1
:10234800743461347434653420346534753420341D
:102358007334633465346C3465347234693473347B
:102368007134753465342034663465346C346934BA
:102378007334203469346D347034653472346434A1
:102388006934653474342E342034503465346C34F4
:102398006C3465346E347434653473347134753424
:1023A80065342034733469347434203461346D34C2
:1023B80065347434203470346F3472347434743443
:1023C800693474346F347234203465346734653456
:1023D80074342E34203455347434203476346534CF
:1023E8006E3465346E346134743469347334203433
:1023F800743465346C346C34753473342034693413
:102408006E3420346D346534743475347334203448
:10241800763475346C34703475347434613474348F
:1024280065342034653475342E34203449346E34A0
:10243800203461346C3469347134753461346D34EA
:102448002034733465346D3420346634723469341E
:102458006E34673469346C346C34613420347534C8
:10246800743420346D346F347234623469342E34E9
:1024780020344834613462346934743461346E34DD
:10248800743420346D346F347234623469342034D7
:10249800743472346934733474346934713475340F
:1024A80065342034733465346E346534633474347D
:1024B8007534733420346534743420346E346534A0
:1024C80074347534733420346534743420346D3482
:1024D80061346C3465347334753461346434613414
:1024E8002E3420344D3461347334733461342034E1
:1024F80076346934743461346534203474346F3418
:10250800723474346F347234203463346F346E34FC
:10251800643469346D3465346E34743475346D34B0
:1025280020346C346134633469346E346934613412
:102538002034713475346934733420347634653416
:102548006C342034653472346F347334203464341A
:102558006F346E34653463342E3420345434653427
:102568006C346C3475347334203469346E34743498
:1025780065346734653472342034663465347534B0
:1025880067346934613474342034733463346534A3
:102598006C34653472346934733471347534653429
:1025A80020347634613472346934753473342034A9
:1025B8006D346F34723462346934203465346E3467
:1025C80069346D3420346E3475346E346334203499
:1025D8006634613475346334693462347534733401
:1025E800203461342E3420344C34693462346534F8
:1025F80072346F3420346A347534733474346F34FD
:1026080020346C3461346F34723465346534743416
:102618002034733469347434203461346D3465344F
:1026280074342034633475347234733475347334C9
:102638002034733469347434203461346D3465342F
:1026480074342034643469346334743475346D34C8
:102658002E340034533465346D3470346534723438
:10266800203461347534633474346F3472342034F4
:102678006E34653471347534653420347634693495
:102688007434613465342034743465346D34703492
:10269800753473342E3420345134753469347334BA
:1026A8002034723469347334753473342034733499
:1026B800653464342034763475346C34703475344D
:1026C800743461347434653420346F346434693458
:1026D8006F34203475347434203465346E3469347E
:1026E8006D342E3420344E3475346C346C3461348B
:1026F800203466346134633469346C346934733437
:10270800693420346D346F3472346234693420345F
:10271800743465346D3470347534733420346934EA
:102728006134633475346C34693473342E34203432
:10273800543469346E3463346934643475346E34B3
:10274800743420346E3475346E3463342034703409
:1027580075346C34763469346E34613472342034B0
:10276800733461347034693465346E3420346534BC
:10277800743420346C346934673475346C3461349F
:10278800203475346C346C3461346D3463346F3494
:1027980072347034653472342E34203456346934CB
:1027A8007434613465342034733475347334633469
:1027B80069347034693474342034743465346C3456
:1027C8006C347534733420346D3461347534723438
:1027D80069347334203461342034643469346134A6
:1027E8006D3420346D3461346534633465346E344B
:1027F800613473342034733465346434203465347C
:102808006E3469346D342E34203450346F3472345D
:1028180074347434693474346F34723420346C34DE
:1028280065346F342034613420346434693461345D
:102838006D34203473346F346C346C3469346334DD
:10284800693474347534643469346E3420347434BF
:1028580065346D3470346F347234203469346434C0
:102868002E3420344534743420346D3461346C345F
:1028780065347334753461346434613420346634B7
:1028880061346D34653473342034613463342034F6
:102898007434753472347034693473342034653464
:1028A80067346534733474346134733420346D346C
:1028B80061346534633465346E34613473342E3472
:1028C800203441347434203465346C3465346D34C8
:1028D80065346E34743475346D342034653475342D
:1028E800203466346134633469346C346934733445
:1028F80069347334203473346534643420346F3469
:10290800643469346F3420346D346F347234623413
:102918006934203471347534693473342034633441
:102928006F346D346D346F3464346F342E34203426
:102938004534673465347334743461347334203403
:1029480064347534693420346934643420346F3421
:1029580072346E34613472346534203461347234C4
:102968006334753420346F34643469346F342034FC
:10297800753474342034733465346D3420346E34D3
:1029880075346C346C346134203470346834613498
:10299800723465347434723461342E3420344D34D6
:1029A8006134753472346934733420347234683461
:1029B8006F346E3463347534733420346134653461
:1029C8006E34653461346E342034763465346C3456
:1029D800203465346C34693474342034733463348B
:1029E80065346C34653472346934733471347534D5
:1029F800653420346D346134753472346934733419
:102A08002034703465346C346C3465346E3474340A
:102A180065347334713475346534203470347534E6
:102A28006C34763469346E346134723420347034E2
:102A380065346C346C3465346E3474346534733492
:102A48007134753465342E34203445346734653434
:102A5800743420346E3475346E34633420347334F3
:102A6800633465346C346534723469347334713466
:102A78007534653420347634693476346534723488
:102A88007234613420346D3461347534723469348D
:102A98007334203469346E34203461346C346934CE
:102AA8007134753461346D342034733465346D3465
:102AB8002E3420344534673465347434203461341A
:102AC8006C346934713475346534743420346E343C
:102AD8006934623468342034703472346134653453
:102AE800733465346E347434203474347234693415
:102AF80073347434693471347534653420346D3406
:102B0800613467346E3461342E34203443346F3486
:102B18006E347334653471347534613474342034EC
:102B280069346E34743465347234643475346D3495
:102B38002034763461347234693475347334203413
:102B4800733469347434203461346D3465347434C6
:102B580020346D34613474347434693473342034FB
:102B6800763475346C347034753474346134743438
:102B78006534203465346E3469346D3420346E34F1
:102B880075346C346C346134203461346C34693499
:102B980071347534653474342E3420344D346134D2
:102BA8007334733461342034763469347434613462
:102BB8006534203474346F34723474346F3472343E
:102BC800203463346F346E34643469346D3465345E
:102BD8006E34743475346D3420346C346134633439
:102BE80069346E346934613420347134753469342D
:102BF80073342E34203444347534693420346134C9
:102C08006334633475346D34733461346E34203412
:102C1800733469347434203461346D3465347434F5
:102C280020346E3475346C346C346134203466343A
:102C38006134633469346C346934733469342034EE
:102C48006D346F34723462346934203474346534CA
:102C58006D347034753473342E3400344E34653426
:102C6800713475346534203463346F346E3476349B
:102C780061346C346C3469347334203461342034F6
:102C880063347234613473342034733465346D348E
:102C98007034653472342034613475346334743478
:102CA8006F34723420346E3465347134753465345D
:102CB800203476346934743461346534203474349F
:102CC80065346D347034753473342034713475342C
:102CD80061346D342E34203451347534693473348E
:102CE800203469347034733475346D34203473345B
:102CF80075347334703465346E34643469347334C1
:102D080073346534203475346C34743472346934F3
:102D18006334653473342034673472346134763400
:102D28006934643461342034643469346334743409
:102D380075346D34203466347534733463346534D3
:102D4800203475347434203470346C346134633412
:102D580065347234613474342E342034413472341E
:102D680063347534203461346334203474346F34FC
:102D7800723474346F347234203464346934673490
:102D88006E3469347334733469346D342034633485
:102D98006F346E34763461346C346C346934733423
:102DA8002034613465346E34653461346E342034D3
:102DB80065347434203474346F34723474346F343A
:102DC8007234203461347434203472346934733486
:102DD800753473342E342034453467346534743490
:102DE800203464346F346C346F34723420346D346E
:102DF8006F3472346234693420346E346F346E3414
:102E08002034613472346334753420347234693454
:102E180073347534733420347134753469347334CD
:102E28002034763461347234693475347334203420
:102E38007134753461346D342E34203443346F3436
:102E48006E3473346534633474346534743475346F
:102E580072342034613464346934703469347334BE
:102E6800633469346E346734203465346C346934BF
:102E78007434203475347434203461346C346934D7
:102E88007134753461346D3420347034753472346F
:102E980075347334203473346934743420346134B1
:102EA8006D346534743420346C347534633474345C
:102EB800753473342E342034503475347234753488
:102EC8007334203469346E3420346D346F346C3488
:102ED8006C346934733420346E3475346E3463342E
:102EE80020347334653464342034693464342E34C3
:102EF800203450346F347334753465347234653427
:102F080020346D346F3472346234693420346C3454
:102F180065346F342034753472346E34613420343F
:102F28006D346F346C346534733474346934653497
:102F38002034613474342E34203443346F346E3486
:102F4800733465346334743465347434753472346A
:102F580020346C3469346234653472346F3420340C
:102F680069346434203466346134753463346934C4
:102F780062347534733420346E34693473346C3489
:102F88002034743469346E34633469346434753489
:102F98006E347434203465346734653474342034C2
:102FA8006E3475346C346C3461346D3420346E3462
:102FB8006F346E3420346E346934733469342E348B
:102FC800203456346134723469347534733420349F
:102FD800643475346934733420346134743420347F
:102FE80063346F346E3473346534633474346534E5
:102FF80074347534723420346C346F3472346534FC
:103008006D342E34203450346F3472347434743444
:10301800693474346F34723420346C3465346F34EA
:103028002034613420346434693461346D3420349C
:1030380073346F346C346C34693463346934743485
:103048007534643469346E342034743465346D34C2
:1030580070346F3472342E342034503475347234F2
:1030680075347334203469346E3420346D346F34DD
:103078006C346C346934733420346E3475346E3483
:1030880063342034733465346434203469346434EC
:103098002034733465346D347034653472342034BC
:1030A80072346934733475347334203469346E344B
:1030B8002E34203445346C34693474342034653407
:1030C8006734653474342034673472346134763448
:1030D8006934643461342034633475346D34203495
:1030E80073346F34633469346934733420346E3420
:1030F800613474346F347134753465342034703409
:1031080065346E34613474346934623475347334BC
:103118002E3420344D346134753472346934733448
:103128002034633475347234733475347334203412
:103138006D346134743474346934733420346D34C8
:103148006F346C34653473347434693465342034C2
:103158006134203469346134633475346C346934CF
:1031680073342034613474342034653472346134F7
:1031780074342034703465346C346C3465346E3493
:103188007434653473347134753465342E342034B2
:103198005634613472346934753473342034763477
:1031A80065346C3420347034683461347234653476
:1031B8007434723461342034763465346C34203499
:1031C80074347534723470346934733420346E3422
:1031D80075346E346334203465346734653474343C
:1031E8002E3420344E3465347134753465342034CB
:1031F800653467346534733474346134733420341B
:1032080063346F346E346734753465342034713404
:1032180075346934733471347534653420346534E5
:1032280067346534733474346134733420346434EB
:10323800693461346D34203469346E342E3400348A
:1032480049347034733475346D34203466346134E1
:1032580075346334693462347534733420347634A5
:103268006934743461346534203461346C346934BD
:10327800713475346534743420346E346534633491
:10328800203475346C346C3461346D3463346F3489
:10329800723470346534723420347334693474345D
:1032A800203461346D3465347434203472346934B4
:1032B80073347534733420346E3475346C346C3430
:1032C80061346D342E34203449346E3474346534AA
:1032D8007234643475346D34203463346F346E342E
:1032E80073346534633474346534743475347234C7
:1032F80020346C3469346234653472346F34203469
:103308006934643420346634613475346334693420
:103318006234753473342E3420344434753469344B
:1033280073342034613474342034743465346C3428
:103338006C34753473342034613474342034753407
:1033480072346E3461342E34203455346C346C3419
:1033580061346D3463346F3472347034653472346C
:103368002034733469347434203461346D346534F2
:1033780074342034723469347334753473342034BB
:103388006E3475346C346C3461346D342034653487
:103398006734653474342034663465346C34693485
:1033A8007334203465346734653474342E342034EF
:1033B80041347234633475342034663465346C3483
:1033C80069347334203462346934623465346E3459
:1033D800643475346D342034753474342034743462
:1033E80072346934733474346934713475346534BF
:1033F8002034653474342034653467346534733468
:1034080074346134733420347134753469347334EA
:10341800203469347034733475346D342E34203468
:10342800523468346F346E346334753473342034F2
:1034380064346F346C346F347234203470347534BF
:1034480072347534733420346E346F346E342034EF
:1034580065346E3469346D342E342034563469340E
:103468007634653472347234613420346F34723493
:1034780063346934203473346134673469347434A0
:1034880074346934733420346534753420347634B4
:103498006F346C347534743470346134743420345B
:1034A8006F34643469346F3420346634613463347F
:1034B80069346C34693473346934733420346D344A
:1034C8006134753472346934733420347334693434
:1034D8007434203461346D34653474342E342034BB
:1034E80055347434203463346F346E347334653433
:1034F80071347534613474342034733465346D3404
:1035080070346534723420347634693476346534F2
:1035180072347234613420346E3461346D34203442
:103528006C3469346234653472346F3420346A34EC
:103538007534733474346F3420346C3461346F34BC
:1035480072346534653474342034733469347434B3
:103558002E342034413420347334633465346C346D
:103568006534723469347334713475346534203495
:10357800703475347234753473342034733465346C
:103588006D3470346534723420346534673465348E
:1035980074342E3420344634723469346E346734CB
:1035A80069346C346C3461342034753474342034A8
:1035B8006D346F347234623469342034743469344D
:1035C8006E3463346934643475346E34743420343E
:1035D80061347534673475346534203469346E3435
:1035E800743465347234643475346D34203476340C
:1035F80065346C3469347434203465347534693412
:1036080073346D346F346434203469346E34203448
:10361800703465346C346C3465346E3474346534A9
:1036280073347134753465342E3420345034653431
:103638006C346C3465346E3474346534733471347A
:103648007534653420346434693461346D3420341D
:1036580076346F346C347534743470346134743443
:10366800203463346F346D346D346F3464346F34A4
:1036780020347334653464342E342034563465343D
:103688006C34693474342034653475346934733473
:103698006D346F346434203469346E3420347034BB
:1036A80065346C346C3465346E3474346534733416
:1036B80071347534653420346D3461347334733443
:1036C8006134203470346C3461346334653472345A
:1036D8006134743420346434753469347334203478
:1036E80075346C34743472346934633469346534D1
:1036F800733420346C346134633475347334203457
:0A3708007334653464342E34003449
:103B8E00FE0012001E00FE0BC82D0034953480344A
:103B9E002E3493345A348C3432349634EC348F348D
:103BAE0024349934FC348434C434883407340834CF
:103BBE0003340234013406340534043420000E126A
:103BCE00BD01BE01F12D20008E158E110130BD07F5
:103BDE000030BE3D3908BB003808BA00BA35BB0DFF
:103BEE00BA35BB0DBA35BB0D3E08803ABC003B085A
:103BFE00803A3C02031D052E3A083D02031C082E96
:103C0E00092EEA2D20008E168E120800F100F20108
:103C1E00F301F201F3017108F0007208303E8600E4
:103C2E0087010108FF3E890A1D2EF036890B1C2ED6
:103C3E007018222E252E20000E16272E20000E1272
:103C4E008E158E110130F2070030F33D7308803A65
:103C5E00F00080307002031D362E08307202031CF5
:103C6E00392E3A2E122E0800210019159911191607
:103C7E0099168C1624008C16210095131E169E1272
:103C8E001E179E130E1523000E1521001D119D15D6
:103C9E001D169D121D131D148E120E128E11230051
:103CAE008E112100951295158B168B17083020005A
:103CBE00B8000030B9009D31E5259E3121009D14DC
:103CCE009D186A2E6B2E672E1C082000BF00C001A7
:103CDE003F08F9004008FA008C1A762E772E652ED2
:103CEE0041084204031D7C2E7D2E652E0830B8003F
:103CFE000030B9009D31E5259E312000C301C4017D
:103D0E00FB01FC010130C5070030C63D0030460204
:103D1E00083003194502031C952E962E982EC501C8
:103D2E00C6013230C1000030C200652E80317928C4
:103D3E00F200052FFC30FF2F6030FF2FDA30FF2FFF
:103D4E00F230FF2F6630FF2FB630FF2FBE30FF2F21
:103D5E00E030FF2FFE30FF2FF630FF2FEE30FF2F1B
:103D6E003E30FF2F1A30FF2F9C30FF2F7A30FF2F5F
:103D7E009E30FF2F8E30FF2FBC30FF2F2E30FF2FA7
:103D8E006E30FF2F2030FF2F7830FF2FF830FF2FAF
:103D9E00AE30FF2F3C30FF2F1C30FF2FA830FF2FEF
:103DAE002A30FF2FEC30FF2F3A30FF2FCE30FF2F6F
:103DBE00E630FF2F0A30FF2F1E30FF2F3830FF2F37
:103DCE007C30FF2F5430FF2F7630FF2F1230FF2F15
:103DDE000230FF2F1030FF2FC630FF2F4030FF2F45
:103DEE004430FF2FF030FF2F0130FF2F2130FF2FF7
:103DFE004130FF2FCB30FF2F0030FF2F7208F00025
:103E0E00F1017108003A03190D2F032F7008203AA3
:103E1E000319032F013A0319FF2E033A0319F72E44
:103E2E00053A0319F52E0F3A0319BB2E013A031961
:103E3E00F92E053A0319C92E013A0319EF2E033A4A
:103E4E000319FB2E1E3A0319A12E013A0319A32EB4
:103E5E00033A0319A52E013A0319A72E073A03199F
:103E6E00A92E013A0319AB2E033A0319AD2E013ACE
:103E7E000319AF2E0F3A0319B12E013A0319B32EBF
:103E8E00023A0319FD2E063A0319ED2E023A0319D2
:103E9E00012F7E3A0319B52E033A0319B72E013AB4
:103EAE000319BB2E073A0319BD2E013A0319BF2E73
:103EBE00033A0319C12E013A0319C32E0F3A0319FF
:103ECE00C72E013A0319A32E033A0319CD2E013A38
:103EDE000319CF2E073A0319D32E013A0319D52E03
:103EEE00033A0319D92E013A0319A12E1F3A0319C9
:103EFE00DD2E013A0319DF2E033A0319E12E013AA2
:103F0E000319AB2E073A0319E32E013A0319E72ED4
:103F1E00033A0319E72E013A0319E92E0F3A031952
:103F2E00C72E013A0319EB2E033A0319A52E013AB7
:103F3E000319BB2E063A0319F92E023A0319F12E74
:103F4E003E3A0319B52E033A0319B72E013A031957
:103F5E00B92E073A0319BD2E013A0319BF2E033AA3
:103F6E000319C12E013A0319C32E0F3A0319C52E98
:103F7E00013A0319C92E033A0319CB2E013A03193C
:103F8E00CF2E073A0319D12E013A0319D52E033A33
:103F9E000319D72E013A0319DB2E1F3A0319DD2E12
:103FAE00013A0319DF2E033A0319E12E013A0319E0
:103FBE00AB2E073A0319E32E013A0319E52E033A05
:103FCE000319E52E013A0319E92E0F3A0319C72EEC
:103FDE00013A0319A92E033A0319A52E013A031922
:103FEE00BB2E063A0319F92E853A0319F32E032F29
:023FFE000800B9
:020000040001F9
:04000E00A4C9CFDFD3
:00000001FF
